:020000003528A1
:100008009300030894000B1110181328A3308100E3
:100018000F08861D920403108F0D0318101414087E
:100028008300930E130E090006158616C32091301F
:1000380023020319B62BA130230203197C2BA2300B
:1000480023020319992B123023020319282B10308D
:10005800230203192E2B1430230203191F2B2323E9
:100068001A280630650018306600831664008E3042
:100078006200831220308B008B1386018501851561
:10008800051406161011861D4C28BD2086197928DE
:1000980006108515051464008E306200861D5728E9
:1000A800BD208619792805195C2885185E284728F7
:1000B8008518472806148B13C32008308D000616B0
:1000C80008306600B72006160310910C03186F2835
:1000D80008306600712818306600B7208D0B672835
:1000E80018306600B72006104728B7200310920D75
:1000F800A330810001308F0001308E001010920172
:100108008B17061410188D280F080E060319882857
:100118008A1B8B13051D8E28851C8E280E08120538
:10012800003803199E288511851898288515851C7F
:100138009B28A428051005199F280514051DA22829
:1001480003108E0D031C86288B1306104728920176
:1001580008308D00B72086190310861D0314920CF1
:100168008D0BAE28080016308C0000008C0BB928C7
:1001780008000C308C0000008C0BBF28080091018F
:1001880064008E30620008308D008518D628051D61
:10019800C92885110310910C851CD02885158D0B55
:1001A800C92808000519C92805100314910C051D54
:1001B800DB2805148D0BC928080064008E30620006
:1001C80008308D00851CE628051DE6280310920CD2
:1001D8000318F72805100519EF280514051DF2283E
:1001E8008D0BE628FF2885118518F8288515851CAC
:1001F800FB288D0BE628851CFF28051DFF28080015
:100208008501860106306500183066001A215A21DA
:100218000130180203191529023018020319182988
:100228000A29060831210A295A210A2901306500BC
:10023800640005181C296400051C1F291830950046
:100248009801013033215A21180895005A21A53008
:100258001802031D1A29A530312998000830970083
:10026800051064000B308100051C3829150896001C
:100278000000960B3C2996000030980C031C4A2974
:1002880065000130960B452965005129650001304C
:100298004D294E29960B4B296500970B3A291508CD
:1002A80096000000960B5529640008000830970056
:1002B800051064000B308100051C602915089600A4
:1002C800003065000130960B662965006B296C29A2
:1002D8006D29960105186E29960A16081502051C3F
:1002E8007029980C970B6D29051878296400080067
:1002F80000306600073099009A018601990A083093
:100308001902031D892999019A0A19088207932954
:10031800A029AD29BA29C729D429E129EE29FF3016
:100328001A02031D9F299B0A03301B02031D9F29E4
:100338009B01013086068229FF301A02031DAC2971
:100348009C0A08301C02031DAC299C010230860659
:100358008229FF301A02031DB9299D0A06301D02A1
:10036800031DB9299D01043086068229FF301A022F
:10037800031DC6299E0A0B301E02031DC6299E01B5
:10038800083086068229FF301A02031DD3299F0AE6
:100398000C301F02031DD3299F01103086068229C5
:1003A800FF301A02031DE029A00A04302002031DB1
:1003B800E029A001203086068229FF301A02031D99
:1003C800ED29A10A17302102031DED29A1014030B2
:1003D80086068229FF301A02031DFA29A20A09306B
:1003E8002202031DFA29A2018030860682290E34D2
:1003F800113411341134113411340E3404340C34E2
:1004080004340434043404340E340E341134013406
:100418000234043408341F340E34113401340634E1
:10042800013411340E34023406340A3412341F34C1
:10043800023402341F3410341E34013401341134B0
:100448000E340E34113410340E34113411340E3489
:100458001F340134013402340234043404340E34B9
:10046800113411340E34113411340E340E34113465
:1004780011340F34013411340E340034003408348C
:1004880004340234003400340234043408340034B0
:100498000034003400340034003400340E34113495
:1004A80011341F341134113411341F341134113400
:1004B80011341134113411340E341E341134113402
:1004C8001134113411341E34113411341E341134E2
:1004D80011341E34103410341034103410341034E5
:1004E8001F34103410341C34103410341F341034BA
:1004F80010341C34103410341034013401340134F5
:100508000134013411340E341134103413341134DD
:1005180011340E34113411341134153413340E34AB
:10052800113410340E34013411340E3411341034B3
:100538001034103411340E340434043404340434C4
:1005480004340E341134123414341834143412347C
:1005580011341B3415341134113411341134193455
:10056800153413341134113411340A340434043476
:1005780004341E34113411341E341134113411343E
:10058800113411340A3404340A3411341134113456
:10059800113415341B3411341F340134023404343B
:1005A800083410341F340434043404340434043458
:1005B800043407308C00B92804308C00B9287E3404
:1005C80030346D34793433345B345F3470347F3491
:1005D800733477341F344E343D344F3447348612E5
:1005E80000000608A300861608000611000023086C
:1005F800860006150800003066002D3086000611BA
:100608002408860000000615061008008614061146
:1006180000002608860006150000061100002708BD
:100628008600061500000611000028088600061539
:10063800000086100800C320230886001A288617A1
:10064800061F242B8613080000306600C3202308E9
:1006580086001A28FF3066000608A300E1201A2841
:10066800A70DA70DA80DA70DA80DA70DA80D0F3054
:10067800A70508000430A600A8012908A70034230C
:100688002A088C0006160000A401FF220A23FF3066
:10069800660023232510F322FE3023020319582B6A
:1006A8002514AB01AC010800F3222308AB00230892
:1006B800A900F3222308AC002308AA008C038C08A5
:1006C80003197B2B2030A607031C6E2BA70A031CDB
:1006D8006E2BA80AAA08031D752B20302902031CBB
:1006E800462B2030A902031C662BAA03662B0800A0
:1006F800A601A801C3202308A7003423A401FF22D0
:100708000A23FF3066002323F322883023020319CB
:10071800912BA301E12006161A2808308C00F32239
:10072800E1208C0B912B06161A28C3202308A90058
:10073800C3202308AA003E232B08A300E1202C088D
:10074800A300E120251CAB2B061625101A28F3223E
:1007580023088C00E1208C0AF322E1208C0BB02BBB
:1007680006161A28C3202308A900C3202308AA00B4
:100778003E232B08A300E1202C08A300E120251C20
:10078800C82B061625101A28F32223088C00E1200E
:100798008C0A0C08AB07031CD22BAC0A1D308C004A
:1007A800F322E120AB03031CDC2BAC030318EF2B73
:1007B8008C0BD42B06162030A607031CE72BA70AA0
:1007C800031CE72BA80AA401FF220A23FF306600B6
:0A07D80020308C00D42B06161A28DE
:1042000000000000000000000000000000000000AE
:10421000000000000000000000000000000000009E
:10422000000000000000000000000000000000008E
:10423000000000000000000000000000000000007E
:10424000000000000000000000000000000000006E
:10425000000000000000000000000000000000005E
:10426000000000000000000000000000000000004E
:10427000000000000000000000000000000000003E
:084000007F007F007F007F00BC
:02400E00FD3F74
:02FFFE0084007D
:00000001FF
